:020000040800F2
:100000005809002045010008FD100008651000088F
:10001000F9100008B1010008AF2E00080000000030
:100020000000000000000000000000007125000832
:10003000F50D00080000000011210008BD27000890
:100040005F0100085F0100085F0100085F01000810
:100050005F0100085F0100085F0100085F01000800
:100060005F0100085F0100085F0100085F010008F0
:100070005F0100085F0100085F0100085F010008E0
:100080005F0100085F0100085F0100085F010008D0
:100090005F0100085F0100085F0100085F010008C0
:1000A0005F0100085F0100085F0100085F010008B0
:1000B0005F010008252800085F0100085F010008B3
:1000C0005F0100085F0100085F0100085F01000890
:1000D0005F010008052A0008612A0008452B000876
:1000E0005F0100085F0100085F0100085F01000870
:1000F0005F0100085F0100085F0100085F01000860
:100100005F0100085F0100085F0100085F0100084F
:100110005F0100085F0100085F0100085F0100083F
:100120005F0100085F0100085F0100085F0100082F
:10013000DFF80CD000F02AF800480047B52F00087F
:10014000580900200648804706480047FEE7FEE7BA
:10015000FEE7FEE7FEE7FEE7FEE7FEE7FEE7FEE777
:10016000C127000831010008D2B201E000F8012BDC
:10017000491EFBD270470022F6E710B513460A4627
:1001800004461946FFF7F0FF204610BD064C074D08
:1001900006E0E06840F0010394E807009847103457
:1001A000AC42F6D3FFF7C8FFEC3200080C3300086E
:1001B00000BFFEE710B502460B460020002104E018
:1001C000545C0444E0B24C1CE1B29942F8DBC443F5
:1001D000E0B2441CE0B210BDFEB5002000900190DA
:1001E000029000F059FF414800780A281DD140488C
:1001F000007840490978884217D13D4840783D4908
:100200004978884211D13A48007A3A49097A8842B5
:100210000BD13748407A3749497A884205D1364868
:10022000008840F40040344908803348008800F4D6
:100230000040002858D0012002F068FE00202F491D
:10024000087048708870C87008712D49087048702F
:100250008870C87008712B49087048708870C87021
:1002600008712949087048708870C870087100F0DA
:1002700013FF0020224908701D48007948701C486F
:10028000407988701A488079C8701948C079087117
:1002900000201E4908701A48407848701848807835
:1002A00088701748C078C870154800790871012017
:1002B00001F0C8F912484078040611488078050416
:1002C0000F48C0780602601930440D490979471873
:1002D00001200F49087000F0DFFE00F0DDFE002075
:1002E0000249087004490880FEBD00000900002092
:1002F000CC0100200C0000200A0000202C0000206F
:100300001600002034000020390000201B000020CF
:100310004100002010B588B07F480078012838D10E
:1003200000207D490870FC207C490870112048702D
:100330007B48007888707A484078C8707848807820
:1003400008717748C078487175480079887107212D
:100350007248FFF72FFF7149C8710020714908608A
:10036000FF22E121012001F021FE08236B4AA82190
:10037000012001F0DDFD012001F064F901206A494E
:10038000C1F8A4016949087000206949088000F09B
:1003900083FE6748008840F6B83188427BDC00F075
:1003A0007BFE604884380068002857D100F074FE56
:1003B0006946012001F09AFD0446204602F026F924
:1003C0005CA002F02DF904F040004028EDD100209F
:1003D0008DF80A000721684600F00DFD55A002F0D7
:1003E0001FF99DF801004E490978884254D19DF8C3
:1003F00002004B49497888424ED19DF80300484994
:100400008978884248D19DF804004549C9788842D6
:1004100042D19DF805004249097988423CD14348C0
:10042000007801281BD141480078401C3F490870E2
:1004300012203A49487007213848FFF7BBFE374978
:10044000C8710020374908600823344AA8210120D8
:1004500001F06EFD01203449C1F8A40158E00020EC
:10046000324908700E21344800F0C5FC31A002F07A
:10047000D7F832480178012001F03EF910202E49CA
:1004800048700E212C4802F0B5F82DA002F0C8F8F3
:10049000012008B010BD16E000202249086011209C
:1004A0001E49487007211D48FFF784FE1B49C8718B
:1004B00008230A46A821012001F03AFD01201A492B
:1004C000C1F8A40124E00020154908704870887024
:1004D000C87008711B49087048708870C87008712E
:1004E0001949087048708870C870087117490870F9
:1004F00048708870C870087130200F4948700E210C
:100500000D4802F077F812A002F08AF80120C0E747
:1005100000F0C2FD0020BCE73E00002042000020A9
:100520002C000020A4812142008021428200002072
:10053000200000200A000000C00300202A00002044
:100540004F4B0A00390000201B000020160000203D
:10055000333030300A00000010B588B04F480088B2
:1005600040F2DC51884278DA4D480068002875D1A5
:1005700000F092FD6946012001F0B8FC044604F049
:10058000400040287CD100208DF80A0007216846F1
:1005900000F031FC43A002F043F89DF8010078B967
:1005A0009DF8020060B99DF8030048B900203E495B
:1005B000087048708870C8700871012008B010BDBC
:1005C0003A480078072803D0384800780D280FD122
:1005D0000020354908709DF8000048709DF8010022
:1005E00088709DF80200C8709DF80300087145E00E
:1005F0002E480078082810D19DF801002A4908707B
:100600009DF8020048709DF8030088709DF8040072
:10061000C8709DF80500087130E02448007809286A
:1006200003D0224800780E2819D100201E490870F6
:100630009DF8010080F0530048709DF8020080F0A2
:10064000430088709DF8030080F04400C8709DF856
:10065000040080F05800087110E014E010E0002061
:10066000114908709DF8010048709DF802008870DB
:100670009DF80300C8709DF80400087101209DE7F3
:1006800000F00AFD08E000200749087048708870F3
:10069000C8700871012091E700208FE73200002028
:1006A000208121420A000000390000202A00002099
:1006B00010B500F0F1FCFE480078082829D1FD486B
:1006C0000078752825D1FB484078702821D1F94859
:1006D000807864281DD1F748C078612819D1F54881
:1006E0000079742815D1F3484079652811D100208C
:1006F000EF49087000BFF048006800F4E060EF497F
:100700000843001DEC490860BFF34F8F00BF00BFD6
:10071000FEE7E8480078752807D0E6480078FA2810
:1007200003D00020E249087010BDE14800780E288F
:1007300000DAF9E7DE480078401EDE49085CFB2855
:1007400000D0F1E7DB48807AA02804D1D8480078AF
:10075000152800D0E8E7D64800780E281ED1D548E5
:100760000078FA2814D1D348407BFB2810D1D44814
:10077000008840F40040D24908800020CC4908702D
:100780000E21CC4800F037FBCEA001F049FF4AE033
:100790000020C7490870CA49088044E0C44800786E
:1007A00015281ED1C3480078FA2814D1C148007D0D
:1007B000FB2810D1C248008840F40040C04908809E
:1007C0000020BB4908701521BA4800F014FBBDA0F9
:1007D00001F026FF27E00020B5490870B8490880DD
:1007E00021E0B348007811281DD1B2480078FA28DA
:1007F00014D1B048007CFB2810D1B148008840F4E7
:100800000040AF4908800020A94908701121A9487B
:1008100000F0F1FAABA001F003FF04E00020A449CE
:100820000870A7490880A648008800F40040002806
:1008300071D000F031FC9F488079A34988719D48B0
:10084000C179A148C1719B48017A9F4801729948BA
:10085000417A9D4841729748807A9B498872084640
:1008600080799A4988719848C1799848C1719648A9
:10087000017A964801729448417A944841729248AC
:10088000807A94284CD018DC732834D00CDC2528CE
:1008900025D004DC21281AD022287DD11BE026286F
:1008A00021D07128F9D122E0742828D075282AD0C7
:1008B00078282CD08228F0D12EE0A03809286BD2DD
:1008C000DFE800F0329CA0F5F4F3F2F1F000002034
:1008D0007D498872CBE100207B498872C7E1002006
:1008E00079498872C3E1002077498872BFE100200E
:1008F00075498872BBE1002073498872B7E1002016
:1009000071498872B3E100206F498872AFE100201D
:100910006D498872ABE1AEE100206B498872A6E1B7
:10092000002069498872A2E1002061490870664888
:100930008079674988716448C1796548C1716248A6
:10094000017A634801726048417A614841725E48A9
:10095000807A5F4988725748407B5B4948735548A5
:10096000817B594881735348C17B5748C1735148B3
:10097000017C554801744F48417C534841744D48AF
:10098000407B544908704B48807B48704948C07B85
:1009900088704848007C00E068E1C8704548407CA9
:1009A000087101204C49087000204C490880012042
:1009B00000F048FE4AA001F033FE04E0FFF7AAFC75
:1009C000044604B100E0F9E700BF45A001F028FEAD
:1009D00000204549087048708870C8700871434904
:1009E000087048708870C870087141490870487074
:1009F0008870C87008713449887238E10020324923
:100A0000887234E13948407848B93848807830B93C
:100A10003648C07818B93548007900B927E1002078
:100A20002349087028488079324988712648C1795D
:100A30003048C1712448017A2E4801722248417A17
:100A40002C4841722048807A2A4988720120C87255
:100A500006200873002048732448017825488173D4
:100A6000224841782348C173204881782148017485
:100A70001E48C1781F4841741C4801791D48817483
:100A8000162101F0B7FD322002F040FA1621194874
:100A900000F0B1F90BA001F0C3FD0020134908706C
:100AA000487029E099E0DDE0D8E0D3E02BE029E0D0
:100AB00003000020040100200CED00E00000FA0516
:100AC000040000200A000000F80200209402002028
:100AD000C00300202C0000203E0000202000002049
:100AE000303030300A000000390000201B000020A8
:100AF000160000205C0300208870C87008715F49F0
:100B00008872B4E0B3E000205D4908705D48017868
:100B1000012000F0F1FD00205B4908805BA001F09E
:100B20007FFD04E0FFF718FD044604B100E0F9E79B
:100B300000BF56A001F074FD504880795549887176
:100B40004E48C1795348C1714C48017A51480172ED
:100B50004A48417A4F4841724848807A4D498872E4
:100B60000120C87206200873002048734A480178A3
:100B700048488173484841784648C173464881785F
:100B8000444801744448C17842484174424801795C
:100B900040488174162101F02DFD322002F0B6F993
:100BA00016213C4800F027F939A001F039FD00205A
:100BB0003949087048708870C870087137490870E2
:100BC00048708870C870087135490870487088701E
:100BD000C87008712949887249E03248407B294928
:100BE000087026488079304988712448C1792E4898
:100BF000C1712248017A2C4801722048417A2A4862
:100C000041721E48807A28498872012048700E215E
:100C1000254801F0EFFC322002F078F919480078FD
:100C20002249088001F0AEFC00201B490870487082
:100C30008870C87008711949087048708870C87049
:100C400008711749087048708870C87008710B499E
:100C500088720CE000200949887208E000200749EA
:100C6000887204E000200549887200E000BF00BFE0
:100C700000200F49088000BF56E50000F802002060
:100C8000030000202A0000203200002034343434D5
:100C90000A0000005C030020390000201B00002037
:100CA0001600002004010020240400202C05002050
:100CB00004000020FA204A490870102048700020E3
:100CC000887000214648C17001714171002044497B
:100CD000887100214248C17101724172002040496F
:100CE000C87400213E480175FB203D494875FA2033
:100CF0003C49087010204870002088700021394855
:100D0000C170017141710020364988710021354858
:100D1000C171017241720020324981F84B000021FB
:100D2000304880F84C10FB202E4981F84D00FA2005
:100D30002D490870102048700020887000212A4832
:100D4000C170017141710020274988710021264836
:100D5000C1710172417200202349C87200212248EA
:100D60000173FB2020494873FA20204908701020A5
:100D700048700020887000211C48C17001714171C9
:100D800000201A49887100211848C171017241720E
:100D900000201649C874002114480175FB2013492E
:100DA0004875FA2012490870102048700020887099
:100DB00000210F48C1700171417100200C498871F8
:100DC00000210B48C1710172417200200849C872AC
:100DD000002107480173FB20054948737047000054
:100DE00094020020F8020020240400205C0300206C
:100DF000C003002070472DE9F04104460E460DE087
:100E00002578281100F030F9074601F0FFFB28464D
:100E100000F02AF9074601F0F9FB641C301EA6F128
:100E20000101CEB2ECD1BDE8F081000030B504463E
:100E300004254FF4302000F06FF80546042D17D13B
:100E40000C48006940F002000A4908610846446104
:100E5000006940F0400008614FF4302000F05CF879
:100E600005460448006941F6FD71084001490861E2
:100E7000284630BD0020024004200B49C96801F01B
:100E8000010109B101200EE00749C96801F0040120
:100E900009B1022007E00449C96801F0100109B155
:100EA000032000E00420704700200240034800694E
:100EB00040F08000014908617047000000200240B6
:100EC00070B504460D460426F00200F025F80646EB
:100ED000042E11D10948006940F00100074908615A
:100EE0002580F00200F018F806460448006941F633
:100EF000FE71084001490861304670BD0020024083
:100F00000248034948600348486070472301674529
:100F100000200240AB89EFCD00B502460423FFF765
:100F2000ABFF034603E0FFF7A7FF0346521E012B6A
:100F300001D1002AF7D102B90523184600BD2DE9D9
:100F4000F04102460025002600200023002400274F
:100F500091F803C00CF00F0591F803C00CF0100CD1
:100F6000BCF1000F03D091F802C04CEA050591F8DE
:100F700000C0BCF1000F31D0146800202BE04FF00E
:100F8000010C0CFA00F3B1F800C00CEA03069E4213
:100F900020D183004FF00F0C0CFA03F7BC4305FA85
:100FA00003FC4CEA040491F803C0BCF1280F06D1FD
:100FB0004FF0010C0CFA00FCC2F814C00AE091F8E2
:100FC00003C0BCF1480F05D14FF0010C0CFA00FC36
:100FD000C2F810C0401C0828D1D31460B1F800C07A
:100FE000BCF1FF0F34DD546800202EE000F1080C46
:100FF0004FF0010808FA0CF3B1F800C00CEA030640
:101000009E4221D183004FF00F0C0CFA03F7BC4332
:1010100005FA03FC4CEA040491F803C0BCF1280F64
:1010200005D100F1080C08FA0CF8C2F8148091F808
:1010300003C0BCF1480F07D100F1080C4FF00108C4
:1010400008FA0CF8C2F81080401C0828CED354606F
:10105000BDE8F081416170470161704701460A882F
:1010600090B2704700BFFEE70146002001F00F027A
:10107000092A04DC01F00F0202F1300003E001F064
:101080000F023732D0B270474CF6CC4001490860AD
:10109000704700000030004010B500F013F810BD9C
:1010A00070B505460C4645F2555000F01FF828462D
:1010B00000F010F8204600F013F800F003F8FFF7F6
:1010C000E3FF70BD4AF6AA2001490860704700009E
:1010D0000030004001494860704700000030004087
:1010E00001498860704700000030004001490860F5
:1010F000704700000030004000BFFEE7704700006E
:101100007CB5054612A103C9CDE900010821284696
:1011100001F006FA05236A463021284600F008FF50
:1011200005236A461021284600F072FE002406E0DE
:101130001DF80400A52800D003E0601CC4B2052CF3
:10114000F6DB00BF052C01D001207CBD0020FCE7B0
:10115000A5A5A5A5A500000008B501211C2000F04B
:10116000E9FF4020ADF8000010208DF803000320B7
:101170008DF8020069463248FFF7E1FE4021304811
:10118000FFF76AFF1020ADF8000069462D48FFF711
:10119000D6FE10212B48FFF75FFF8020ADF800003E
:1011A00048208DF8030003208DF80200694624488A
:1011B000FFF7C5FE4FF40070ADF8000010208DF869
:1011C000030003208DF8020069461D48FFF7B7FEB3
:1011D0004FF400711A48FFF73FFF4FF48050ADF80D
:1011E000000069461648FFF7AAFE4FF480511448E4
:1011F000FFF732FF4FF48070ADF8000048208DF803
:10120000030003208DF8020069460D48FFF797FEA2
:1012100001F0B4F801F070F800200B4908600120DB
:101220000A49C1F89001002007490C3108600120EB
:101230000749C1F8B0010821002001F071F908BD8B
:10124000000C014000080140988121420000214229
:101250000080214210B5044602222321204600F0DE
:10126000A5FE05231E4A2A21204600F061FE052323
:101270001B4A3021204600F05BFE3F222121204600
:1012800000F094FE01222221204600F08FFE1A2257
:101290002521204600F08AFE24222621204600F047
:1012A00085FE0F222021204600F080FE0A223121F7
:1012B000204600F07BFE01223D21204600F076FE14
:1012C00000223C21204600F071FE7022272120469A
:1012D00000F06CFEFF22E221204600F067FE10BD08
:1012E000A932000810B5044602222321204600F04E
:1012F0005DFE04231E4A2A21204600F019FE042325
:101300001B4A3021204600F013FE302221212046C6
:1013100000F04CFE01222221204600F047FE12225E
:101320002521204600F042FE24222621204600F0FE
:101330003DFE0F222021204600F038FE08223121F8
:10134000204600F033FE01223D21204600F02EFE13
:1013500000223C21204600F029FE70222721204651
:1013600000F024FEFF22E221204600F01FFE10BD07
:10137000E032000810B5044602222321204600F086
:1013800015FE04231E4A2A21204600F0D1FD042325
:101390001B4A3021204600F0CBFD3022212120467F
:1013A00000F004FE01222221204600F0FFFD282249
:1013B0002521204600F0FAFD0C222621204600F0CF
:1013C000F5FD0F222021204600F0F0FD06223121FC
:1013D000204600F0EBFD01223D21204600F0E6FD15
:1013E00000223C21204600F0E1FD7022272120460A
:1013F00000F0DCFDFF22E221204600F0D7FD10BD09
:10140000D632000810B5044602222321204600F0FF
:10141000CDFD04231E4A2A21204600F089FD042325
:101420001B4A3021204600F083FD30222121204636
:1014300000F0BCFD01222221204600F0B7FD33223E
:101440002521204600F0B2FD04222621204600F08E
:10145000ADFD0F222021204600F0A8FD09223121F8
:10146000204600F0A3FD01223D21204600F09EFD14
:1014700000223C21204600F099FD702227212046C1
:1014800000F094FDFF22E221204600F08FFD10BD08
:10149000CC32000810B5044602222321204600F079
:1014A00085FD05231E4A2A21204600F041FD052323
:1014B0001B4A3021204600F03BFD3F2221212046DF
:1014C00000F074FD01222221204600F06FFD12225F
:1014D0002521204600F06AFD04222621204600F046
:1014E00065FD0F222021204600F060FD0A223121F7
:1014F000204600F05BFD01223D21204600F056FD14
:1015000000223C21204600F051FD70222721204678
:1015100000F04CFDFF22E221204600F047FD10BD07
:101520009A32000810B5044602222321204600F01A
:101530003DFD05231E4A2A21204600F0F9FC052323
:101540001B4A3021204600F0F3FC302221212046A6
:1015500000F02CFD01222221204600F027FD12225E
:101560002521204600F022FD21222621204600F0E0
:101570001DFD0F222021204600F018FD0A223121F6
:10158000204600F013FD00223D21204600F00EFD14
:1015900001223C21204600F009FD7022272120462F
:1015A00000F004FDFF22E221204600F0FFFC10BD08
:1015B0008B32000810B5044601222321204600F09A
:1015C000F5FC05231E4A2A21204600F0B1FC052324
:1015D0001B4A3021204600F0ABFC3022212120465E
:1015E00000F0E4FC01222221204600F0DFFC192259
:1015F0002521204600F0DAFC04222621204600F0B6
:10160000D5FC0F222021204600F0D0FC06223121FB
:10161000204600F0CBFC01223D21204600F0C6FC14
:1016200000223C21204600F0C1FC702227212046E8
:1016300000F0BCFCFF22E221204600F0B7FC10BD08
:10164000B832000810B504461CB9002027490860CC
:1016500003E0002025490C310860012223212046A7
:1016600000F0A4FC0323224A2A21204600F060FC5B
:101670000323204A3021204600F05AFC0122212178
:10168000204600F093FC01222221204600F08EFC2F
:101690002A222521204600F089FC0422262120460A
:1016A00000F084FC0F222021204600F07FFC06225F
:1016B0003D21204600F07AFC01223C21204600F02A
:1016C00075FC70222721204600F070FCFF22E221E9
:1016D000204600F06BFC1CB901200449086003E0BF
:1016E000012002490C31086010BD000098812142A0
:1016F000813200087C32000870B504460D461CB9E2
:1017000000203649086003E0002034490C310860AD
:10171000132D57D2DFE805F00A0E12161A1E2226E4
:101720002A2E32363A3E42464A4E52002046FFF7B3
:10173000F9FE47E0204600F093FA43E0204600F02F
:101740001FFB3FE02046FFF7A5FE3BE0204600F0F0
:10175000F7F937E0204600F0D3F833E02046FFF7F2
:1017600079FD2FE0204600F0A3F92BE0204600F0A1
:10177000BFFA27E02046FFF71DFF23E0204600F0D8
:101780002FF81FE0204600F023FA1BE0204600F06F
:101790006FF817E02046FFF735FE13E02046FFF70D
:1017A00009FF0FE02046FFF7E5FD0BE0204600F0C3
:1017B00037F907E02046FFF795FD03E0204600F0EB
:1017C000E7F800BF00BF1CB901200449086003E02E
:1017D000012002490C31086070BD0000988121424F
:1017E00010B5044602222321204600F0DFFB04232B
:1017F0001E4A2A21204600F09BFB04231B4A30216D
:10180000204600F095FB30222121204600F0CEFB3F
:1018100001222221204600F0C9FB2022252120465A
:1018200000F0C4FB20222621204600F0BFFB0F223F
:101830002021204600F0BAFB08223121204600F08A
:10184000B5FB01223D21204600F0B0FB00223C21E7
:10185000204600F0ABFB70222721204600F0A6FBBB
:10186000FF22E221204600F0A1FB10BDBD3200089E
:1018700010B5044602222321204600F097FB0423E2
:101880001E4A2A21204600F053FB04231B4A302124
:10189000204600F04DFB30222121204600F086FB3F
:1018A00001222221204600F081FB12222521204620
:1018B00000F07CFB24222621204600F077FB0F223B
:1018C0002021204600F072FB0A223121204600F040
:1018D0006DFB01223D21204600F068FB00223C21E7
:1018E000204600F063FB70222721204600F05EFBBB
:1018F000FF22E221204600F059FB10BDC73200084C
:1019000010B5044602222321204600F04FFB052398
:101910001E4A2A21204600F00BFB05231B4A3021DA
:10192000204600F005FB30222121204600F03EFB3E
:1019300001222221204600F039FB122225212046D7
:1019400000F034FB24222621204600F02FFB0F223A
:101950002021204600F02AFB0A223121204600F0F7
:1019600025FB01223D21204600F020FB00223C21E6
:10197000204600F01BFB70222721204600F016FBBA
:10198000FF22E221204600F011FB10BDA432000826
:1019900010B5044602222321204600F007FB042351
:1019A0001E4A2A21204600F0C3FA04231B4A302194
:1019B000204600F0BDFA30222121204600F0F6FA40
:1019C00001222221204600F0F1FA1422252120468E
:1019D00000F0ECFA04222621204600F0E7FA0F225C
:1019E0002021204600F0E2FA0A223121204600F0B0
:1019F000DDFA01223D21204600F0D8FA00223C21E8
:101A0000204600F0D3FA70222721204600F0CEFABB
:101A1000FF22E221204600F0C9FA10BDE53200089D
:101A200010B5044602222321204600F0BFFA042309
:101A30001E4A2A21204600F07BFA04231B4A30214B
:101A4000204600F075FA30222121204600F0AEFA3F
:101A500001222221204600F0A9FA12222521204647
:101A600000F0A4FA24222621204600F09FFA0F223B
:101A70002021204600F09AFA08223121204600F069
:101A800095FA01223D21204600F090FA00223C21E7
:101A9000204600F08BFA70222721204600F086FABB
:101AA000FF22E221204600F081FA10BDDB3200085F
:101AB00010B5044601222321204600F077FA0523C1
:101AC0001E4A2A21204600F033FA05231B4A302102
:101AD000204600F02DFA30222121204600F066FA3F
:101AE00001222221204600F061FA10222521204601
:101AF00000F05CFA04222621204600F057FA0F225B
:101B00002021204600F052FA06223121204600F022
:101B10004DFA01223D21204600F048FA00223C21E6
:101B2000204600F043FA70222721204600F03EFABA
:101B3000FF22E221204600F039FA10BDAE32000843
:101B400010B5044602222321204600F02FFA052377
:101B50001E4A2A21204600F0EBF905231B4A3021BA
:101B6000204600F0E5F930222121204600F01EFA3F
:101B700001222221204600F019FA122225212046B6
:101B800000F014FA24222621204600F00FFA0F223A
:101B90002021204600F00AFA08223121204600F0D8
:101BA00005FA01223D21204600F000FA00223C21E6
:101BB000204600F0FBF970222721204600F0F6F9BC
:101BC000FF22E221204600F0F1F910BD9F3200080B
:101BD00010B5044602222321204600F0E7F9042331
:101BE0001E4A2A21204600F0A3F904231B4A302173
:101BF000204600F09DF930222121204600F0D6F940
:101C000001222221204600F0D1F91C222521204664
:101C100000F0CCF924222621204600F0C7F90F223B
:101C20002021204600F0C2F908223121204600F090
:101C3000BDF901223D21204600F0B8F900223C21E7
:101C4000204600F0B3F970222721204600F0AEF9BB
:101C5000FF22E221204600F0A9F910BDC23200089F
:101C600010B5044603222321204600F09FF90523E6
:101C70001E4A2A21204600F05BF905231B4A302129
:101C8000204600F055F93F222121204600F08EF930
:101C90003F222221204600F089F9282225212046D2
:101CA00000F084F904222621204600F07FF90B225F
:101CB0002021204600F07AF90A223121204600F046
:101CC00075F901223D21204600F070F900223C21E7
:101CD000204600F06BF970222721204600F066F9BB
:101CE000FF22E221204600F061F910BD9032000889
:101CF00010B5044601222321204600F057F90323A2
:101D00001E4A2A21204600F013F903231B4A3021E2
:101D1000204600F00DF930222121204600F046F93E
:101D200001222221204600F041F92A2225212046C5
:101D300000F03CF904222621204600F037F90F225A
:101D40002021204600F032F907223121204600F000
:101D50002DF900223D21204600F028F901223C21E6
:101D6000204600F023F970222721204600F01EF9BA
:101D7000FF22E221204600F019F910BDB33200081D
:101D800010B5044603222321204600F00FF9052355
:101D90001E4A2A21204600F0CBF805231B4A302199
:101DA000204600F0C5F830222121204600F0FEF840
:101DB00001222221204600F0F9F810222521204698
:101DC00000F0F4F804222621204600F0EFF80F225C
:101DD0002021204600F0EAF80A223121204600F0B6
:101DE000E5F801223D21204600F0E0F800223C21E8
:101DF000204600F0DBF870222721204600F0D6F8BC
:101E0000FF22E221204600F0D1F810BD95320008F3
:101E10002DE9F0478046894615461E46B8F1000F69
:101E200016D10020174908604946404600F024FBBF
:101E30000746002406E0FF21404600F01DFB285520
:101E4000601CC4B2B442F6DB01200E49086015E004
:101E500000200D4908604946404600F00DFB07464A
:101E6000002406E0FF21404600F006FB2855601CD8
:101E7000C4B2B442F6DB0120034908603846BDE82D
:101E8000F087000090012142B081214270B50546E3
:101E90000E4685B90020114908603146284600F0F9
:101EA000EBFAFF21284600F0E7FA044601200C492E
:101EB000C1F890010FE000200A4908603146284629
:101EC00000F0DAFAFF21284600F0D6FA0446012095
:101ED0000549C1F8B001204670BD000090012142C3
:101EE00000002142B08121420080214270B50646A7
:101EF0000D461021304600F013FB07213046FFF756
:101F0000C5FF044622462721304600F04FF804F072
:101F1000400050B10A232A4661213046FFF778FF7E
:101F2000FF22E221304600F041F8204670BD00005B
:101F30002DE9F0478046894615461E46B8F1000F48
:101F400016D10020174908604946404600F094FA2F
:101F50000746002406E015F8011B404600F08CFA05
:101F6000601CC4B2B442F6DB01200E49086015E0E3
:101F700000200D4908604946404600F07DFA0746BA
:101F8000002406E015F8011B404600F075FA601CBD
:101F9000C4B2B442F6DB0120034908603846BDE80C
:101FA000F087000090012142B08121422DE9F041EB
:101FB00004460E46154684B9002011490860314692
:101FC000204600F059FA07462946204600F054FA08
:101FD00001200C49C1F890010FE000200A49086077
:101FE0003146204600F048FA07462946204600F0D0
:101FF00043FA01200549C1F8B0013846BDE8F08137
:102000009001214200002142B08121420080214202
:1020100008B54FF4C06000F071F826208DF800007C
:1020200001208DF8010002208DF8020001208DF8BA
:102030000300684600F02AF827208DF800000120F0
:102040008DF801008DF802008DF80300684600F05D
:102050001DF825208DF8000000208DF801000120DA
:102060008DF802008DF80300684600F00FF81D207F
:102070008DF8000000208DF801008DF8020001208D
:102080008DF80300684600F001F808BD70B5002126
:1020900000230F22C47804B3154C246804F4E064D0
:1020A000C4F5E064210AC1F10403CA40447804FA8B
:1020B00003F184781440214309010E4C0678A155A0
:1020C000047804F01F050124AC4005786D11AD00C3
:1020D00005F1E025C5F8004109E0047804F01F058A
:1020E0000124AC40044D0678761145F8264070BDB9
:1020F0000CED00E000E400E080E100E00249014373
:10210000024A1160704700000000FA050CED00E083
:102110007047000029B1064AD2690243044BDA61D4
:1021200004E0034AD2698243014BDA617047000040
:102130000010024029B1064A92690243044B9A6199
:1021400004E0034A92698243014B9A6170470000A0
:102150000010024070B5012144F20D00FFF7EAFFC4
:1021600001210220FFF7D6FF042000F013FB1249E3
:10217000B1F1807F00D31DE021F07F40401E4FF081
:10218000E022506150170F22002807DA13071D0EB6
:102190000A4B00F00F04241F1D5503E013071C0E0B
:1021A000074B1C5400BF00204FF0E0229061072035
:1021B000106100BF70BD000080A9030018ED00E0B1
:1021C00000E400E070B50021002300240022002577
:1021D0002C4E766806F00C0121B1042905D008299F
:1021E00021D105E0284E066020E0274E06601DE064
:1021F000244E766806F47013224E766806F4803416
:10220000022606EB93431CB9204E5E43066009E0AC
:102210001C4E7668C6F34046751C1B4EB6FBF5F6A1
:102220005E43066002E0184E066000BF00BF154E18
:10223000766806F0F0010909154E725C0668D64012
:102240004660104E766806F4E061090A104E725C32
:102250004668D64086600B4E766806F46051C90A1F
:102260000B4E725C4668D640C660064E766806F431
:102270004041890B074E725CC668B6FBF2F60661F8
:1022800070BD00000010024000127A0000093D00FD
:10229000880000209800002010B586B0002414218A
:1022A00001A8FDF768FF0A2201A9084800F012F80A
:1022B00000BF07E001A810F81400054A02F8140056
:1022C000601CC4B20A2CF5DB06B010BD0000030888
:1022D0004005002070B504460D461646002300BF99
:1022E00007E02046FEF7BAFE25F81300A41C581C90
:1022F000C3B2B342F5DB70BD00B587B0012141F236
:102300000500FFF717FFE020ADF8180018208DF842
:102310001B0003208DF81A0006A91648FEF70FFED1
:10232000E0211448FEF798FE0020ADF804004FF4B9
:102330008270ADF806000020ADF80800ADF80A0084
:10234000ADF80C004FF40070ADF80E001820ADF899
:1023500010000020ADF812000720ADF8140001A90C
:10236000054800F06BF80121034800F04DF807B074
:1023700000BD0000000801400030014000B587B0FA
:1023800001218803FFF7C6FE01210920FFF7D2FED5
:102390004FF46040ADF8180018208DF81B000320A2
:1023A0008DF81A0006A91648FEF7C9FD4FF46041E2
:1023B0001348FEF751FE0020ADF804004FF4827080
:1023C000ADF806000020ADF80800ADF80A00ADF841
:1023D0000C004FF40070ADF80E001820ADF810009E
:1023E0000020ADF812000720ADF8140001A905483F
:1023F00000F024F80121034800F006F807B000BD02
:10240000000C01400038004021B1028842F0400237
:10241000028004E002884FF6BF731A4002807047C2
:102420000246002013890B400BB1012000E0002080
:1024300070470146888970478181704710B5002236
:10244000028802F441520B884C8823438C88234332
:10245000CC8823430C8923434C8923438C89234311
:10246000CC8923431A430280838B4FF2FF742340AD
:1024700083830B8A038210BD2DE9F04106460F4687
:1024800026BB06E0601CC4B2C82C02DB0020BDE8FD
:10249000F08102212048FFF7C3FF0028F2D039461F
:1024A0001D48FFF7C9FF002405E0601CC4B2C82C1A
:1024B00001DB0020EBE701211748FFF7B1FF0028FF
:1024C000F3D01548FFF7B5FFC5B222E005E0601C68
:1024D000C4B2C82C01DB0020D9E702210F48FFF766
:1024E0009FFF0028F3D039460C48FFF7A5FF0024D2
:1024F00005E0601CC4B2C82C01DB0020C7E7012145
:102500000648FFF78DFF0028F3D00448FFF791FF3E
:10251000C5B22846BBE7000000300140003800404B
:1025200070B505460C467DB90F4800884FF6C77157
:1025300008400D4908800846008820430880012192
:102540000A48FFF761FF0EE0084800884FF6C771A0
:102550000840064908800846008820430880012179
:102560000248FFF751FF70BD0030014000380040C5
:10257000704770B504460D4629462046FEF7A0FC7C
:1025800070BD000010B586B00024142101A8FDF72D
:10259000F2FD00BF07E00B4830F8140001A921F854
:1025A0001400601CC4B20A2CF5DB074800F0EAF8FE
:1025B0000A2201A9044800F009F800F07AFC06B0EC
:1025C00010BD00002C050020000003082DE9F0419B
:1025D00005460F461646002400BF07E037F81410E2
:1025E0002846FFF7C6FFAD1C601CC4B2B442F5DB41
:1025F000BDE8F08170B504460D46034A29462046E1
:1026000000F028F870BD00000038014010B5044605
:102610000249204600F00EF810BD000000440040C2
:1026200010B504460249204600F02DF810BD000008
:102630000044004070B504460D4600BF8021284686
:1026400000F064FB0028F9D02146284600F02BFC5E
:10265000012070BD2DE9F04104460D46164614B91F
:102660000120BDE8F0810AE014F8017B31463846CC
:10267000FFF7E0FF08B90020F3E7681E85B2002DE0
:10268000F2D10120EDE770B504460E460CB90120E9
:1026900070BD11E014F8015B0A2D06D131460D2002
:1026A000FFF7C8FF08B90020F2E731462846FFF7D8
:1026B000C1FF08B90020EBE720780028EAD101200B
:1026C000E6E710B500F002F810BD00000CB50020E0
:1026D000019000902A48006840F480302849086042
:1026E00000BF2748006800F4003000900198401CAB
:1026F0000190009818B90198B0F5A06FF1D1204869
:10270000006800F4003010B10120009001E00020CA
:1027100000900098012831D1194840681849486054
:102720000846406848600846406848600846406877
:1027300020F47C1048600846406840F498104860D7
:102740000846006840F08070086000BF0C480068D0
:1027500000F000700028F9D00948406820F003001C
:10276000074948600846406840F00200486000BFE2
:102770000348406800F00C000828F9D10CBD0000A7
:102780000010024010B50446FEF7BAFB2046FEF7E3
:102790004DFB10BD042808D14FF0E021096941F03C
:1027A00004014FF0E022116107E04FF0E0210969D8
:1027B00021F004014FF0E0221161704770470000E2
:1027C00010B51448006840F001001249086008463E
:1027D0004068114908400F494860084600680F49A1
:1027E00008400C4908600846006820F48020086012
:1027F0000846406820F4FE0048604FF41F008860DF
:102800000020C862FFF75DFF4FF0006004490860D8
:1028100010BD0000001002400000FFF8FFFFF6FEB0
:1028200008ED00E010B50121204800F07EF80028F6
:102830003AD001211D4800F069F81D480088401C6D
:102840001B4908801B480088401C1A4908801A4808
:102850000088401C1849088018480078C0B14FF41F
:1028600000711748FEF7F8FB16480088401C154910
:10287000088008460088B0F5C87F09DB4FF4007176
:102880000F48FEF7E7FB00200E4908800B4908704F
:102890000948008841F28831884202D10020064967
:1028A000088001200849087010BD000000040040A5
:1028B00020000020320000202200002025000020FF
:1028C0000010014026000020240000203EB50546EF
:1028D0000C4601210220FFF71DFCADF80450ADF8B5
:1028E00000400020ADF80600ADF802006946064839
:1028F00000F036F801221146034800F027F80121C4
:10290000014800F006F83EBD00040040CA430282C0
:10291000704721B1028842F00102028004E002887F
:102920004FF6FE731A400280704730B50246002011
:1029300000230024158A05EA0103958905EA0104AC
:1029400013B10CB1012000E0002030BD1AB1838921
:102950000B43838102E083898B43838170470000AE
:10296000002202881D4B98420ED01D4B98420BD07E
:10297000B0F1804F08D01B4B984205D01A4B9842BB
:1029800002D01A4B984204D14FF68F731A404B88ED
:102990001A43174B984207D0164B984204D04FF673
:1029A000FF431A40CB881A4302808B8883850B88AB
:1029B00003850A4B98420BD0094B984208D00E4B26
:1029C000984205D00D4B984202D00D4B984201D150
:1029D0000B7A03860123838270470000002C01409C
:1029E000003401400004004000080040000C00409A
:1029F000001000400014004000400140004401402D
:102A00000048014010B540F22551124800F08BF902
:102A100088B140F225510F4800F0CFF80D4800F082
:102A20003DFAC4B20C480D49097844540B4800786B
:102A3000401C0A4908700821064800F067F901287F
:102A400006D10821034800F0AFF8024800F026FA4A
:102A500010BD0000003801400401002003000020E8
:102A600010B540F22551124800F05DF988B140F2EE
:102A700025510F4800F0A1F80D4800F00FFAC4B23C
:102A80000C480D49097844540B480078401C0A4909
:102A900008700821064800F039F9012806D10821FC
:102AA000034800F081F8024800F0F8F910BD00007A
:102AB00000440040EC0400208500002010B586B0E2
:102AC000044601210520FFF735FB01214804FFF7EB
:102AD00021FB0420ADF8140003208DF81600182007
:102AE0008DF8170005A91548FEF729FA0820ADF85A
:102AF000140004208DF8170005A91048FEF71FFAEE
:102B000001940020ADF80800ADF80A00ADF80C0003
:102B1000ADF810000C20ADF80E0001A9084800F037
:102B200051F9012240F22551054800F026F9012112
:102B3000034800F051F806B010BD00000008014045
:102B40000044004010B540F22551144800F0EBF865
:102B5000B0B140F22551114800F02FF80F4800F0B5
:102B60009DF9C4B20E480F49097844540D480078C5
:102B7000401C0C4908700846007800F00F000870EF
:102B80000821064800F0C2F8012806D108210348B0
:102B900000F00AF8014800F081F910BD004800403B
:102BA000CC0100200900002001F40072B2F5007F82
:102BB00000D100BFCA430280704710B50022002335
:102BC00040F66A14A14200D100BF0A1201249440C9
:102BD000A3B2DC43048010BD21B1828942F40052CB
:102BE000828104E082894DF6FF731A40828170472A
:102BF00000B585B0012144F20400FFF79BFA4FF4C1
:102C00000070ADF8000003208DF8020018208DF848
:102C1000030069463948FEF792F94FF48060ADF839
:102C2000000004208DF8030069463448FEF787F958
:102C30004FF4164001900020ADF80800ADF80A00EE
:102C4000ADF80C00ADF810000C20ADF80E0001A995
:102C50002B4800F0B7F8012240F22551284800F037
:102C60008CF801212648FFF7B7FF01218804FFF700
:102C700051FA01210820FFF75DFA4FF48060ADF8AA
:102C8000000003208DF8020018208DF8030069462B
:102C90001C48FEF754F94FF40060ADF80000042022
:102CA0008DF8030069461748FEF749F94FF496502E
:102CB00001900020ADF80800ADF80A00ADF80C0056
:102CC000ADF810000C20ADF80E0001A90E4800F080
:102CD00079F801A90C4800F075F8012240F225515D
:102CE000094800F04AF801210748FFF775FF402125
:102CF0000348FFF759FF05B000BD00000008014080
:102D000000380140000C014000480040024600200D
:102D1000B1F5007F00D100BF13880B400BB101203B
:102D200000E00020704770B5024600240023002513
:102D3000002040F66A16B14200D100BFC1F342152F
:102D400001F01F03012606FA03F3012D02D1968933
:102D5000334006E0022D02D1168A334001E0968A04
:102D600033400C12012606FA04F41688344013B1DD
:102D70000CB1012000E0002070BDF0B50346002436
:102D800000260025002040F66A17B94200D100BF96
:102D90001846C1F3421401F01F06012707FA06F591
:102DA000012C01D10C3004E0022C01D1103000E0E4
:102DB00014301AB107682F43076002E00768AF4379
:102DC0000760F0BD2DE9F04786B005460E460024A9
:102DD000A24600BFA1460027B08900B100BF2F4620
:102DE0002C8A4CF6FF700440F08804432C82AC8996
:102DF0004EF6F3100440B0883189084371890843C6
:102E00000443AC81AC8A4FF6FF400440B0890443D0
:102E1000AC8201A8FFF7D6F91F48874202D1DDF83E
:102E200010A001E0DDF80CA0A88900F4004040B13A
:102E30000AEBCA0000EB0A1031684900B0FBF1F858
:102E400007E00AEBCA0000EB0A1031688900B0FB0A
:102E5000F1F86420B8FBF0F004012009642101FBC3
:102E60001089A88900F4004040B1322000EBC9006D
:102E7000B0FBF1F000F00700044308E0322000EB63
:102E800009106421B0FBF1F000F00F0004432C8125
:102E900006B0BDE8F0870000003801400146888890
:102EA000C0F308007047C1F308028280704700BF7A
:102EB000FEE710B5FDF7FAFF10BD0000014A024918
:102EC00000F013B8392F00089C00002002E008C869
:102ED000121F08C1002AFAD170477047002001E094
:102EE00001C1121F002AFBD170472DE9F04116469F
:102EF0000F460446002503E03946B047641C6D1CAC
:102F000020780028F8D12846BDE8F08110B50246A7
:102F10000BE0C82007E0122101E04B1E99B2002906
:102F2000FBDC431E98B20028F5DC131EA2F101045D
:102F3000A2B2EED110BD000070B504460D46E0B25D
:102F40000549088000BF40210348001FFFF7DEFE4F
:102F50000028F8D0204670BD0438014008B5012192
:102F60001020FFF7E7F80120ADF8000010208DF8E1
:102F7000030003208DF8020069460D48FDF7DFFFCE
:102F800001210B48FEF768F84FF40070ADF800001F
:102F900010208DF8030003208DF8020069460448D4
:102FA000FDF7CDFF4FF400710148FEF753F808BD5F
:102FB00000100140FFF7CEF8FFF72AF840F2712128
:102FC0000420FEF76DF8FEF767F841F61F4109206F
:102FD000FFF77CFCFFF7C2FFFFF70AFE4FF4E1307A
:102FE000FFF76CFDFEF7B8F8FEF756F802E04BA0CD
:102FF000FFF764FF0120FEF783F80028F7D1FDF703
:1030000059FEFEF749F849480068C0434849C1F8ED
:103010008001C820FFF77AFF4548D0F88001C043FF
:103020004349C1F88001062142A0FDF7E4FE43A018
:10303000FFF7F6FAFEF730F841A0FFF73FFF012057
:10304000FEF700FBFFF728F946480078464908706C
:1030500008460078132857D2DFE800F00A0E12164F
:103060001A1E22262A2E32363A3E42464A4E520036
:103070003EA0FFF723FF47E03FA0FFF71FFF43E01D
:1030800040A0FFF71BFF3FE041A0FFF717FF3BE029
:1030900042A0FFF713FF37E043A0FFF70FFF33E035
:1030A00045A0FFF70BFF2FE046A0FFF707FF2BE03F
:1030B00048A0FFF703FF27E049A0FFF7FFFE23E04A
:1030C0004AA0FFF7FBFE1FE04BA0FFF7F7FE1BE057
:1030D0004DA0FFF7F3FE17E050A0FFF7EFFE13E05F
:1030E00052A0FFF7EBFE0FE054A0FFF7E7FE0BE066
:1030F00056A0FFF7E3FE07E058A0FFF7DFFE03E06E
:103100005AA0FFF7DBFE00BF00BF3220FFF7FEFE34
:1031100003E0FDF761F8FDF7CBFAFAE754686520A4
:10312000322E3447204572726F7221008001224294
:103130000000224231323334353600000A000000EC
:103140000A5043B6D4C2EBC8EDBCFECDA8D3C3B081
:10315000E6B1BE56312E392D323031383035313569
:103160000A000000400500202A000020BDADCEF777
:10317000D0ADD2E90D0A0000CCECB2A8D0ADD2E9B6
:103180000D0A0000D4C6C4CFD0ADD2E90D0A0000AC
:10319000B9F3D6DDD0ADD2E90D0A0000CBC4B4A896
:1031A000D0ADD2E90D0A0000C4DAC3C9B9C5D0ADAB
:1031B000D2E90D0A00000000B0B2BBD5D0ADD2E913
:1031C0000D0A0000C9BDCEF7F6CEC5B5D0ADD2E927
:1031D0000D0A000056434F4DB2E2CAD40D0A00005A
:1031E000C1C9C4FEB5E7D0C50D0A0000C1C9C4FEFF
:1031F000D2C6B6AF0D0A00005470D7A8D3C3D0AD65
:10320000D2E90D0A00000000C4DAC3C9B9C5D2C6AC
:10321000B6AFD0ADD2E90D0A00000000B9E3CEF799
:10322000D2C6B6AFD0ADD2E90D0A0000CBC4B4A867
:10323000B5E7D0C5D0ADD2E90D0A0000B8A3BDA84E
:10324000D5E6D7C6D0ADD2E90D0A0000CBD5D6DD84
:10325000C4BEC0BCD0ADD2E90D0A0000D6D8C7ECC0
:10326000D2C6B6AFD0ADD2E90D0A0000C9BDCEF7C7
:10327000D2C6B6AFD0ADD2E90D0A0000344310106B
:1032800001344310100133200D547933200D54794B
:10329000344310100101101043343223ABBA01340F
:1032A00012BBAA0134128675014656431000346ED3
:1032B0004610013443101001862C95010136E4A715
:1032C000BC014218BAE801341286750133200D544E
:1032D00000862C9500005A454E4B00AABB123400C4
:1032E0003412BBAA00254310120000000C33000862
:1032F00000000020A0000000CC2E0008AC33000825
:10330000A0000020605F0000DC2E0008000000002C
:103310000000000000000000D1D1E0D0000000005B
:10332000D2D20000000000000000000000000000F9
:10333000000000000000000000000000000000008D
:10334000000000000000000000000000000031321A
:103350003334353637383931323334353637383916
:1033600000000000000000000000000000003132FA
:1033700033343536373839313233343536373839F6
:10338000000000000000000000000000000000003D
:103390000000000000000000010203040102030419
:0C33A000060708090204060800000000EF
:0400000508000131BD
:00000001FF
